:030000000233CDFB
:0C33CD0078FFE4F6D8FD75815E02341430
:100EC5000A53746172743A20004950436F6E6E651F
:100ED50063745245510A004950436F6E6E656374E1
:100EE500003E432C562C43432CC0E4E0EFF2E5F0E2
:100EF50020D1E8EDEAEEEC49500A003E432C4D4185
:100F0500432C25303262583A25303262583A253022
:100F15003262583A25303262583A25303262583AB0
:100F250025303262582C4D414320E0E4F0E5F10ACA
:100F3500003E432C5645522C20332E3120EEF22014
:100F450025732025732CC2E5F0F1E8FF20495020D8
:100F5500ECEEE4F3EBFF0A00466562203031203207
:100F65003030380031383A30373A3335003E432C8B
:100F75004C442C50524F473A20202020202020203E
:100F8500202020202020202020202020202020205C
:100F9500202020202020202020202020202020204C
:100FA500202020202020202020202020202020203C
:100FB500202020202020202020202020202CC4E0BC
:100FC500F2E020EFF0EEF8E8E2EAE828F4E0E9EBF9
:100FD500290A003E2A2C312CCEF1EDEEE2EDFBE59F
:100FE50020EFE0F0E0ECE5F2F0FB20F1E5F2E5E2E0
:100FF500EEE3EE20E8EDF2E5F0F4E5E9F1E00A00D4
:101005003E412C4130312C2562752E2562752E25E9
:1010150062752E2562752C495020E0E4F0E5F1203B
:10102500E0E4E0EFF2E5F0E00A003E412C41303229
:101035002C2562752E2562752E2562752E25627505
:101045002C495020E0E4F0E5F120EEF1ED2E20F101
:10105500E5F0E2E5F0E00A003E412C4130332C2575
:1010650062752E2562752E2562752E2562752C49B1
:101075005020E0E4F0E5F120F0E5E72E20F1E5F081
:10108500E2E5F0E00A003E412C4130342C25627542
:101095002E2562752E2562752E2562752CCCE0F104
:1010A500EAE020F1E5F2E80A003E412C4130352C1A
:1010B5002562752E2562752E2562752E2562752C85
:1010C500D8EBFEE70A003E532C4130362C256275DD
:1010D5002CC2F0E5ECFF20EEE6E8E42E20EAE2E89B
:1010E500F2E0EDF6E8E820282A3130ECF1290A0093
:1010F5003E2A2C312CC4EEEF2E20EFE0F0E0ECE59B
:10110500F2F0FB20F1E5F2E5E2EEE3EE20E8EDF2A8
:10111500E5F0F4E5E9F1E00A003E422C5330312CCC
:101125002562752CC6E4E0F2FC20E7E0EFF0EEF175
:10113500E020F1EEE5E4E8EDE5EDE8FF20EEF22054
:10114500F1E5F0E2E5F0E00A003E422C5330322CA6
:101155002562752CCEE1ECE5ED20F120F1E5F0E21C
:10116500E5F0EEEC20E1E5E720EAE2E8F2E0EDF675
:10117500E8E90A003E422C5330332C2562752CCF0A
:10118500E5F0E5E7E0EFF3F1EA20EFF0E820EFEE38
:10119500F2E5F0E520F1E2FFE7E820F120F1E5F0E6
:1011A500E2E5F0EEEC0A003E422C5330342C256289
:1011B500752CCDE5F220EFE5F0E5E4E0F7E820E475
:1011C500E8E0E3EDEEF1F2E8EAE820E220F1E5F00F
:1011D500E2E5F00A003E422C5330352C2562752C91
:1011E500CAE0EDE0EB20F8E8F0EEEAEEE2E5F8E043
:1011F500F2E5EBFCEDEEE3EE20EEE1ECE5EDE00AE9
:10120500003E532C5330362C25303262582530326F
:1012150062582530326258253032625825303262A4
:101225005825303262582C4D414320E0E4F0E5F179
:1012350020F8E8F0EEEAEEE2E5F8E0F2E5EBFCEDA9
:10124500EEE3EE20EEE1ECE5EDE00A003E454E442E
:101255000A0044756D705820202020203030203041
:1012650031203032203033203034203035203036B4
:10127500203037203038203039203041203042208E
:1012850030432030442030452030460A003A003AA9
:1012950020000A0044756D70442020202020303045
:1012A500203031203032203033203034203035208A
:1012B500303620303720303820303920304120304A
:1012C500422030432030442030452030460A004536
:1012D5007272206B657900526420656570726F6D5E
:1012E5000A005264204D454D0A00526420436F6444
:1012F500650A0044656275674950204F4E0A0044EF
:10130500656275674950204F46460A004465627517
:101315006755736572204F6E0A004465627567559F
:10132500736572204F46460A0044656275674D73C2
:1013350067204F6E0A0044656275674D7367204FDD
:1013450046460A00436F6E666967206C6F636B21C2
:101355000A00577220656570726F6D0A002053612F
:10136500766520656570726F6D210A004572722081
:101375004D414321004C6F61643E3E002A003C41D3
:1013850030313D003C4130323D003C4130333D0081
:101395003C4130343D003C4130353D003C41303628
:1013A5003D003C21003C5330313D003C5330323D43
:1013B500003C5330333D003C5330343D003C53300A
:0913C500353D003C5330363D007B
:063C9B00010B000109000D
:103D0600C2AFC28E438910758BFF758DB7D2ABD209
:043D16008ED2AF2278
:03001B000232A30B
:1032A300C0E0C083C082C0D0C2AFC28E758BFF7531
:1032B3008DB720060675A61E75A6E10509D202E59F
:1032C3000B6002050BE50AD394014002150A050EB3
:1032D300E50E540F7050D20EE50E543F701AD20013
:1032E30090668DE0601204F0E0D394B4400A9080BD
:1032F300007480F0C2AF80FE906688E0600204F044
:10330300906104E0600214F090668EE0D394014073
:1033130003E014F0300502050CE50DD3946440047A
:10332300D2068002050DE508D3940140021508D2A8
:0C3333008ED2AFD0D0D082D083D0E03258
:1008A400C291C290D2B5C20B7D027C007F07123C7C
:1008B4007E8F24E524646060097D017F60123C36EC
:1008C400D20BE4FDFC7F0B123C7E8F24E52430E642
:1008D400097D04E4FF123C5AD20B7D017C007F07A2
:1008E400123C7E8F24E5247008FD7FFF123C36D233
:1008F4000B300B03126000C2AFC288C2A8C2AA7533
:100904008900123662906341E0B4FA09A3E064CE30
:1009140070030209A4E4F52474392524F582E4342F
:1009240063F583E4F00524E524B443EC9063417457
:10093400FAF0A374CEF0A374CCF0906347740AF079
:10094400E4A3F0A304F0A3F090634C7403F0A37445
:10095400CCF090633D74FFF0A3F0A3F0E4A3F09017
:1009640063587405F0E4F524E5242401FFE433FE20
:1009740074392524F582E43463F583E0FD123CEDFB
:100984000524E524C3944340DFE4F5A775A61E754A
:10099400A6E1907FF0F0A3F09080007480F080FED8
:1009A400D2AF90634C7403F0A374CCF0E490634B27
:1009B400F0123073C2B51236E0C206123AC0906328
:1009C40058E0C3940350037403F0D20BC20DC20C5D
:1009D400D293200B077E0E7FC5122D84E490657898
:1009E400F0123D06C2AFA37408F09062B77424F00D
:1009F400E4A3F0906341E09062B9F0906342E09028
:100A040062BAF0906343E09062BBF0906344E0907C
:100A140062BCF0906345E09062BDF0906346E09064
:100A240062BEF0750A01E490657AF0C207C208C29A
:100A340009C20AD2AF75A70775A61E75A6E1200BD9
:100A440018AF24FE7D03122E85E4FF1231597E6314
:100A54007F78E4FB7D01122F7F90668DE060037444
:100A640001F0E4906104F0A37455F0A37481F0E400
:100A7400F50CE4F50D906104E0700312180690661D
:100A84008EE0B401119080007410F0E490668EF052
:100A9400D20BC20CC20D908008E0F52430E405D2DC
:100AA400077410F0E52430E508D20990800874201A
:100AB400F0E52430E608D2089080087440F0E50C94
:100AC400D394034023908002E4F0908001F090805E
:100AD40000F0E50CD39406400FE4F50CC2039065D6
:100AE4007AF0750A01123AC09080A0E070031237C0
:100AF4005C9080B8E070031237D69080D0E0700329
:100B04001239A0908000E07013300710122B7D90F2
:100B14006334EFF0D394004003120026908002E087
:100B24007006908000E06005D205020A76C205E4F2
:100B3400F50C906104E06003020A76300912122970
:100B44000A906334EFF0D394004005E0FF123D1E99
:100B5400200803020CD5122795906334EFF070033C
:100B6400020A76906378E054BF247F7003020C3845
:100B7400147003020C1024026003020C6B200B0798
:100B84007E0E7FCE122D84300F7920037690635031
:100B9400E07006906354E0605B906684E0FF9063CD
:100BA40050E0B50724906685E0FE906351E0B506F9
:100BB40018906686E0FE906352E0B5060C90668756
:100BC400E0FE906353E06E602B906354E06F7033EB
:100BD400906685E0FF906355E0B50727906686E050
:100BE400FF906356E0B5071B906687E0FF9063575C
:100BF400E0B5070F90657A7401F0123D21750A0182
:100C0400020CD590668474FFF0020CD590668DE0DA
:100C140060037401F090667CE0FF90637AE06F609B
:100C240003020CD590667CE004F0E4F50A90657844
:100C3400F0020CD5300303020CD5906347E0700337
:100C4400020A7612001ED203E4F50A906578F09049
:100C5400668804F0E490667BF0A3F0200B737E0EAC
:100C64007FDC122D84806A90668DE060037401F04D
:100C7400300352906378E020E74B90637AE0FF9072
:100C8400667BE0FE6F600D906683E07007EE146F84
:100C9400703F801390667BE004F0906334E0FFD3F0
:100CA40094044003123D209060007482F0A3740108
:100CB400F090637AE0906002F07E607F007D031222
:100CC40035E2020A76300F0920030690668474FF29
:100CD400F0200303020D8AE50A706B12333FEF60C4
:100CE400207E647F78906479E02404FD1235E290DC
:100CF4006683E06003020A76906358E0F50A020A0C
:100D040076906688E0D3943C403C906683E07036ED
:100D140090668804F09062B6E0702B123D1FE49058
:100D24006478F0A37412F090667CE090647AF0A387
:100D340074FDF090610763A20190647C63A2017F5B
:100D4400121224E3809B123D1AEF60159060007428
:100D540083F0E4A3F07E607F007D021235E2020A94
:100D640076E50A64016003020A76906578E004F08F
:100D7400E0C394055003020CE5C203E490657AF0E5
:100D8400123D21020A76E50A64016003020A7690A4
:100D9400657AE014604624FE6042147003020E7803
:100DA40024046003020A76E4F50C200F1390657A9C
:100DB4007404F0906578E05401F0750A01020A7633
:100DC4009080027410F0E490657AF090657804F0F5
:100DD400750AC890668474FFF0020A76906684E00F
:100DE4007003020E679064787480F090647A7401E2
:100DF400F0E4A3F0A304F0A37430F0A3747BF0E454
:100E0400F524747F2524F582E43464F583747DF03D
:100E140074802524F582E43464F583E4F0E5242425
:100E240007906479F07C667D8490634CE0FAA3E0DB
:100E3400FB7F021234DE7E647F78E5242409FD12F0
:100E440035E2906683E0601B12001ED203E4F50ACB
:100E5400906578F090668804F0E490667BF0A3F0E7
:100E6400020A7690657A7404F0906358E02432F5AF
:100E74000A020A769080027410F0750A039065786D
:100E8400E06401FFF090657A7401F0EF70199063EB
:100E940054E06013FCA3E0FDA3E0FEA3E0FF906632
:100EA40084122096020A76906350E0FCA3E0FDA32E
:100EB400E0FEA3E0FF906684122096020A7680FE8C
:010EC400220B
:10002600906379E0B444047F0180027F0090637896
:10003600E0B447047E0180027E00EE5F604A906372
:1000460041E090637AF0906342E090637BF09063C6
:1000560043E090637CF0906344E090637DF09063AE
:1000660045E090637EF0906346E090637FF0906396
:10007600797452F09062B063A2019080A863A201E5
:100086007F061224E302089A906334E0C394085072
:10009600030208A3906341E0FF90637AE06F600378
:1000A6000208A3906342E0FF90637BE06F60030267
:1000B60008A3906343E0FF90637CE06F600302084F
:1000C600A3906344E0FF90637DE06F60030208A3A2
:1000D600906345E0FF90637EE06F60030208A390A3
:1000E6006346E0FF90637FE06F60030208A39063BE
:1000F60079E0B444159062B0E0B4FF0E63A20190BB
:1001060080A863A2017F061224E390668DE0600357
:100116007401F090668E7464F09063797452F09076
:100126006378E0646D60030202A37BFF7A0E79E6D2
:10013600121C9D7BFF7A0F7900906341E0F52EA398
:10014600E0F52FA3E0F530A3E0F531A3E0F532A307
:10015600E0F533121C9D752EFF752F0F75305D75FA
:1001660031FF75320F7533697BFF7A0F7936121CB2
:100176009D7BFF7A0F7972121C9D7BFF7A0F79D8CF
:10018600121C9D7BFF7A107905906347E0F52EA33C
:10019600E0F52FA3E0F530A3E0F531121C9D7BFFBF
:1001A6007A10792F906350E0F52EA3E0F52FA3E0A7
:1001B600F530A3E0F531121C9D7BFF7A10795D9036
:1001C6006354E0F52EA3E0F52FA3E0F530A3E0F5A8
:1001D60031121C9D7BFF7A10798B90633DE0F52EE2
:1001E600A3E0F52FA3E0F530A3E0F531121C9D7BCB
:1001F600FF7A1079AE906339E0F52EA3E0F52FA3D0
:10020600E0F530A3E0F531121C9D7BFF7A1079CB27
:10021600906358E0F52E121C9D7BFF7A1079F5123B
:100226001C9D7BFF7A11791EA20FE433F52E121C5A
:100236009D7BFF7A11794E906683E0F52E121C9D08
:100246007BFF7A11797990668DE0F52E121C9D7BE5
:10025600FF7A1179AC9062B6E0F52E121C9D7BFFF9
:100266007A1179DAA201E433F52E121C9D7BFF7A0E
:1002760012790690667DE0F52EA3E0F52FA3E0F552
:1002860030A3E0F531A3E0F532A3E0F533121C9D6F
:10029600122C817BFF7A127951121C9D2290637871
:1002A600E0644C70757E127F57122D84906380E057
:1002B600F525A3E0F526E4F5287E127F92122D841B
:1002C6007D03AF26AE25122E857E127F94122D84D5
:1002D600E4F527852682852583E0FF74822527F5A8
:1002E60082E43463F583EFF00526E52670020525E2
:1002F6000527E527B410DC7E637F82E4FB7D1012C0
:100306002F7F7E127F97122D840528E528C394102F
:1003160040A77E127F97122D8422906378E0646C4A
:10032600705CF5297E127F99122D84E4F528AF2999
:100336007E007D03122E857E127F94122D84E4F5B5
:1003460027A829E6FF74822527F582E43463F5831E
:10035600EFF005290527E527B410E67E637F82E4E2
:10036600FB7D10122F7F7E127F97122D840528E5C4
:1003760028C3940840B87E127F97122D842290637A
:1003860078E0644B7061F527746A2527F582E434BA
:1003960063F583E06032746A2527F582E43463F5F9
:1003A60083E0F46023746A2527F582E43463F583D9
:1003B600E0FF74802527F582E43463F583E0B50712
:1003C600100527E527B408C09061047432F00208CE
:1003D6009A9063787421F0300B0302089A7E127F9C
:1003E600D4122D8402089A906378E0B4521A200B36
:1003F600077E127FDC122D849063787472F07E6320
:100406007F787D0812356222906378E064497045F2
:10041600200B077E127FE7122D84906380E0F5257E
:10042600A3E0F526E4F527852682852583E0FF747B
:10043600822527F582E43463F583EFF00526E52669
:10044600700205250527E527B480DC7E637F787D6D
:100456008A12356222906378E064437079A3E0647F
:10046600527046200B077E127FEF122D8490638018
:10047600E0F525A3E0F526E4F52785268285258384
:10048600E493FF74822527F582E43463F583EFF065
:100496000526E526700205250527E527B480DB7EBF
:1004A600637F787D8A12356222906379E0645760B3
:1004B600030208A3906380E0F525A3E0F526748285
:1004C6002527F582E43463AD82FC7B80AF26AE251A
:1004D600123BDC02089A906378E0644460030205EC
:1004E6006D906380E0FF6444700302089AEFB431B4
:1004F6000CC20B7E127FF8122D8402089A9063803C
:10050600E0B4300CD20B7E137F04122D8402089ABD
:10051600906380E0B4320CD20C7E137F11122D84CE
:1005260002089A906380E0B4330CC20C7E137F1FDE
:10053600122D8402089A906380E0B4340CD20D7EAA
:10054600137F2E122D8402089A906380E0B4350C36
:10055600C20D7E137F3B122D8402089A906380E0C1
:10056600FF123D1D02089A906104E07013200B07EC
:100576007E137F49122D849063787421F002089AC5
:100586009061047432F0906378E0FFB4510A908071
:10059600007480F0C2AF80FEEF64577045200B07F1
:1005A6007E137F57122D84906381E0906334F0E4CC
:1005B600F527906334E0FFE527C39F400302089ABE
:1005C60074822527F582E43463F583E0FF90638027
:1005D600E0252724AFF582E43461F583EFF00527A3
:1005E60080D0906378E06453600302069C200B077A
:1005F6007E137F62122D84906341E0FF9061B8E024
:100606006F703C906342E0FF9061B9E06F7030908C
:100616006343E0FF9061BAE0B50724906344E0FFCE
:100626009061BBE0B50718906345E0FF9061BCE0C0
:10063600B5070C906346E0FF9061BDE06F601690D1
:1006460063787421F0300B0302089A7E137F7112CF
:100656002D8402089AE4F527E4F50DAF27FE74AF62
:100666002527F582E43461F583E0FD123CED05278C
:10067600E527C394FE40E19080007480F0C2AFE4A9
:10068600907FF0F0A3F0907FFD74AAF0A374FFF0C2
:10069600A37455F080FE906378E0644F704C9063CD
:1006A60080E0F525A3E0F526E5264525700A200B12
:1006B600077E137F7A122D84200B077E137F81120B
:1006C6002D84E4F52774822527F582E43463F583C7
:1006D600E0852682852583F00526E5267002052518
:1006E6000527E527B480DE02089A906378E0FFB418
:1006F60045279080007480F0906380E0FDA3E09031
:100706007FF0CDF0A3EDF0C2AF907FFD74AAF0A309
:1007160074FFF0A37455F080FEEF64656003020871
:100726009A906380E0FFA3E0907FF0CFF0A3EFF014
:10073600E4F525F526D3907FF1E09526907FF0E04D
:1007460095254020E4F50D2526FFE5253401FE8597
:100756002682852583E0FD123CED0526E5267002FE
:10076600052580D17E137F83123459EF4E60201207
:100776000003906347EFF0120003906348EFF01216
:100786000003906349EFF012000390634AEFF07E96
:10079600137F89123459EF4E602012000390635084
:1007A600EFF0120003906351EFF0120003906352D2
:1007B600EFF0120003906353EFF07E137F8F123435
:1007C60059EF4E6020120003906354EFF0120003BD
:1007D600906355EFF0120003906356EFF01200039A
:1007E600906357EFF07E137F95123459EF4E6020D9
:1007F60012000390633DEFF012000390633EEFF0AA
:1008060012000390633FEFF0120003906340EFF095
:100816007E137F9B123459EF4E60201200039063C3
:1008260039EFF012000390633AEFF0120003906381
:100836003BEFF012000390633CEFF07E137FA112B2
:100846003459EF4E6008123A63906358EFF0E4F5BE
:1008560027E4F50DE5272401FFE433FE7439252747
:10086600F582E43463F583E0FD123CED0527E527C8
:10087600C3944340DC9080007480F0C2AFE4907F64
:10088600F0F0A3F0907FFD74AAF0A374FFF0A374B8
:0D08960055F080FE7E637F787D081235628C
:0108A3002232
:103BA400AE07EEC39430400BEED394395005EE24A7
:103BB400D0FF22EEC39461400BEED394665005EE21
:103BC40024A9FF22EEC39441400BEED39446500542
:083BD400EE24C9FF22AF062216
:103CD3009062AFE004F070069062AEE004F0906290
:0A3CE300AEE0FEA3E0FF123CB722A2
:10000300123CD3123BA4EFC454F0FEC006123CD3FF
:08001300123BA4D0E02FFF22F4
:103A6300E4906A8CF0123CD3906A8DEFF0C39430EB
:103A73004018E0FFD394395011906A8CE02407F585
:103A830082E43461F583EFF08011906A8CE02407BF
:103A9300F582E43461F583E4F0800C906A8CE004F1
:103AA300F0E0D3940840BE752D00752E00752F00ED
:0C3AB300E4F5307B017A6179071225F1FF
:013ABF0022E4
:043459008E2A8F2BFD
:10345D009062AEE4F0A374FFF0123CD3EF606EF413
:10346D00606B852B82852A83E493B507EC752C015F
:10347D00E52B252CF582E4352AF583E49360259020
:10348D0062AFE0252CFF9062AEE03400FE123CB737
:10349D00E52B252CF582E4352AF583E493B5070455
:1034AD00052C80CCE52B252CF582E4352AF583E41B
:1034BD009370A6E52C24FFFFE434FFFE9062AFE08D
:1034CD002FF09062AEE03EF07E007F0122E4FEFF21
:0134DD0022CC
:103073007E137FA7123459EF4E70037F01227E1314
:103083007FAA123459EF4E600C123CD3EF24D024A4
:10309300FF920F8002D20F7E137FB0123459EF4E8E
:1030A300600C123CD3EF24D0906683F08005E4904B
:1030B3006683F07E137FB6123459EF4E600C123CD8
:1030C300D3EF24D090668DF08005E490668DF07E7A
:1030D300137FBC123459EF4E600C123CD3EF24D053
:1030E3009062B6F08005E49062B6F07E137FC21260
:1030F3003459EF4E600C123CD3EF24D024FF9201DD
:103103008002C20190634163A20190667D63A201C4
:103113007F061224E330013B7E137FC8123459EF3C
:103123004E603012000390667DEFF012000390664C
:103133007EEFF012000390667FEFF01200039066BB
:1031430080EFF0120003906681EFF01200039066A7
:0631530082EFF07F002274
:103B1900906579E0C3947C503D906579E0FE04F0AE
:103B290074B72EF582E43462F583EFF0BF0A27906B
:103B39006579E0FF04F074B72FF582E43462F58308
:103B4900E4F0906579E0FF1232039065797408F02A
:073B59009062B8E004F022C5
:103AC0009080007480F090633963A201F583F582E1
:103AD00063A2017F081224E390634163A2019080F6
:103AE0008863A2017F0A1224E3908092E4F0A37419
:103AF00032F0A37401F090634BE0FF9080B1F0903E
:103B000080E1EFF09080957455F0A3F09080007400
:093B100001F090800974F0F0222C
:10375C00908009E04410F09080A0E0706C9080A103
:10376C007482F09080A874FFF0A3F0A3F0A3F07F14
:10377C00039080AEEFF07FCBA3EFF07F039080AC93
:10378C00EFF0A374CBF09080007402F0906A80127A
:10379C0020A200000000906A80E0908040F0906AC7
:1037AC0081E0908041F0906A82E0908042F0906AD3
:1037BC0083E0908043F0A3E4F0A3F0A3F0A3F09097
:0937CC008018F0A3F0A3F0A3F0B3
:0137D50022D1
:1039A000908009E04440F09080D17482F090634CA4
:1039B000E0FF9080DEF090634DE0FF9080DFF090BC
:1039C00080027402F0906A841220A200000000902D
:1039D0006A84E0908058F0906A85E0908059F09079
:1039E0006A86E090805AF0906A87E090805BF0A34E
:1039F000E4F0A3F0A3F0A3F0908030F0A3F0A3F0E4
:023A0000A3F031
:013A020022A1
:1037D600908009E04420F09080B8E0706C9080B949
:1037E6007482F07F039080C6EFF07FCDA3EFF07F69
:1037F600039080C4EFF0A374CDF09080C074FFF006
:10380600A3F0A3F0A3F09080017402F0906A8812EE
:1038160020A200000000906A88E090804CF0906A38
:1038260089E090804DF0906A8AE090804EF0906A30
:103836008BE090804FF0A3E4F0A3F0A3F0A3F09008
:093846008024F0A3F0A3F0A3F02C
:01384F002256
:1034DE008C258D26A907EAFDE975F018A424ACFF0A
:1034EE00E5F034808F82F583EDF0EBFDE975F01891
:1034FE00A4FFAEF024ACFBEE34808B82F583A3EDFB
:10350E00F08526828C83E0FDEF24A8FFEE3480FE4A
:10351E008F82F583EDF08526828C83A3E08F828ED9
:10352E0083A3F0852682852583A3A3E0FDE975F0AC
:10353E0018A424A8FFE5F03480FE8F82F583A3A3A0
:10354E00EDF08526828C83A3A3A3E08F828E83A3C6
:04355E00A3A3F02211
:063562008D2AAB07AA064A
:10356800908000E020E572906A80E0FCA3E0FDA373
:10357800E0FEA3E0F52E8E2D8D2C8C2BAE02AF0332
:103588008E838F8263A201E52D540744C0F583859D
:103598002E8263A201AF2A122555E4FCFDFEE52E1A
:1035A800252AF52EEE352DF52DED352CF52CEC359F
:1035B8002BF52B908040E52BF0A3E52CF0A3E52D0F
:1035C800F0A3E52EF09080007420F0AF2EAE2DAD64
:0935D8002CAC2B906A80122096A5
:0135E10022C7
:0635E2008D25AB07AA06CF
:1035E800908002E020E572906A84E0FCA3E0FDA3ED
:1035F800E0FEA3E0F5298E288D278C26AE02AF03C6
:103608008E838F8263A201E528540744D0F5838511
:10361800298263A201AF25122555E4FCFDFEE529A8
:103628002525F529EE3528F528ED3527F527EC353C
:1036380026F526908058E526F0A3E527F0A3E5288F
:10364800F0A3E529F09080027420F0AF29AE28ADF0
:0936580027AC26906A841220962A
:013661002246
:023159008F25C0
:10315B00908001E030E5037F0022906A88E0FCA3B9
:10316B00E0FDA3E0FEA3E0F5298E288D278C2690A9
:10317B00667D63A201E528540744C8F5838529823F
:10318B0063A2017F0612256BE5292406F529E43598
:10319B0028F528E43527F527E43526F52690657BB9
:1031AB0063A201E528540744C8F58385298263A2ED
:1031BB0001AF2512256BE4FCFDFEE5292525F5293C
:1031CB00EE3528F528ED3527F527EC3526F5269035
:1031DB00804CE526F0A3E527F0A3E528F0A3E5292D
:1031EB00F09080017420F0AF29AE28AD27AC26906B
:0731FB006A88122096AF253F
:0132020022A9
:102B7D009081E0E0F525052505250525052505258B
:102B8D0005250525052505250525908010E0F52849
:102B9D00A3E0F529A3E0F52AA3E0F52B9081E1E070
:102BAD00F5250525052505250525052505250525D8
:102BBD00052505250525908014E0F52CA3E0F52DC0
:102BCD00A3E0F52EA3E0F52FE52EB52A08E52FB5E8
:102BDD002B037F0022E4F525E52E540744E0F58311
:102BED00852F8263A20190637863A2017F0812256D
:102BFD009B90637A63A2019062B063A2017F06127B
:102C0D0024E3906378E0F526A3E0F527E4F525901D
:102C1D006378E0702AA3E024F8F525E52E540744E7
:102C2D00E0F583852F8274082582F582E43583F5DE
:102C3D008363A20190637863A201AF2512259BAE39
:102C4D0026E4FCFDE52F2527F52FE52E3EF52EED8F
:102C5D00352DF52DEC352CF52C908014E52CF0A3AD
:102C6D00E52DF0A3E52EF0A3E52FF0908000744044
:032C7D00F0AF2590
:012C80002231
:102795009081E6E0F5250525052505250525052571
:1027A50005250525052505250525908028E0F5281D
:1027B500A3E0F529A3E0F52AA3E0F52B9081E7E056
:1027C500F5250525052505250525052505250525C4
:1027D50005250525052590802CE0F52CA3E0F52D94
:1027E500A3E0F52EA3E0F52FE4F525E52EB52A0A9D
:1027F500E52FB52B05C2080228EFE52E540744F056
:10280500F583852F8263A20190637863A2017F0817
:1028150012259B906378E0F526A3E0F527E527458B
:102825002670099080027410F07F0022906684E083
:10283500FFF4602D90637AE06F7076906685E0FF17
:1028450090637BE06F706A906686E0FF90637CE042
:102855006F705E906687E0FF90637DE06F60228019
:102865005090637AE0906684F090637BE090668593
:10287500F090637CE0906686F090637DE0906687DB
:10288500F0906378E0702AA3E024F8F525E52E544E
:102895000744F0F583852F8274082582F582E43597
:1028A50083F58363A20190637863A201AF251225A6
:1028B5009BAE26E4FCFDE52F2527F52FE52E3EF5FD
:1028C5002EED352DF52DEC352CF52CAF2BAE2AAD97
:1028D50029AC28AB2FAA2EA92DA82CD312208540D0
:1028E500099080027410F07F002290802CE52CF076
:1028F500A3E52DF0A3E52EF0A3E52FF0908002745B
:0429050040F0AF25CA
:0129090022AB
:10290A009081E3E0F52505250525052505250525FD
:10291A000525052505250525052590801CE0F528B2
:10292A00A3E0F529A3E0F52AA3E0F52B9081E4E0E2
:10293A00F52505250525052505250525052505254D
:10294A00052505250525908020E0F52CA3E0F52D29
:10295A00A3E0F52EA3E0F52FE4F525E52EB52A0A26
:10296A00E52FB52B05C209022A55E52E540744E87E
:10297A00F583852F8263A20190600463A2017F0E12
:10298A001225B1906004E0F526A3E0F52790600CCB
:10299A00E0FFF4604590667DE0FEEF6E706EA3E0A6
:1029AA00FF90600DE06F706490667FE0FF90600EAC
:1029BA00E06F7058906680E0FF90600FE06F704C97
:1029CA00906681E0FF906010E06F7040906682E050
:1029DA00FF906011E06F60048032D2D9906004E009
:1029EA00702AA3E024F2F525E52E540744E8F5837E
:1029FA00852F82740E2582F582E43583F58363A2DE
:102A0A000190600463A201AF251225B1AE26E4FC51
:102A1A00FDE52F2527F52FE52E3EF52EED352DF573
:102A2A002DEC352CF52CAF2BAE2AAD29AC28AB2FCB
:102A3A00AA2EA92DA82CD31220855006E5274526B3
:102A4A0070099080017410F07F0022908020E52C9C
:102A5A00F0A3E52DF0A3E52EF0A3E52FF090800179
:052A6A007440F0AF25EF
:012A6F002244
:042D84008E2A8F2BD9
:102D8800E4F52CF52D908000E030E511052DE52DBA
:102D98007002052CD39488E52C941340E8908000A9
:102DA800E030E503022E84906A80E0FCA3E0FDA3F6
:102DB800E0FEA3E0F5318E308D2F8C2EE531FFE556
:102DC800305407FEE42FF52DEE34C0F52C852D8206
:102DD800F5837423F0052DE52D7002052C532CC7BF
:102DE800F582852C83740AF0052DE52D7002052CDB
:102DF800532CC790634163A201852C83852D826380
:102E0800A2017F061225557406252DF52DE4352CD3
:102E1800F52C852A83852B8263A201852C83852D39
:102E28008263A201122539E4FCFDFE906A80E0F875
:102E3800A3E0F9A3E0FAA3E02FFFEE3AFEED39FD97
:102E4800EC38FCEF2408FFE43EFEE43DFDE43CFCE6
:102E5800906A80122096906A80E0908040F0906A94
:102E680081E0908041F0906A82E0908042F0906A20
:0C2E780083E0908043F09080007420F014
:012E8400222B
:062F7F008E2A8F2B8D2C21
:102F8500E4F52DF52E908000E030E511052EE52EB7
:102F95007002052DD39488E52D941340E8908000A8
:102FA500E030E503023072906A80E0FCA3E0FDA307
:102FB500E0FEA3E0F5328E318D308C2FE532FFE552
:102FC500315407FEE42FF52EEE34C0F52D852E8203
:102FD500F5837423F0052EE52E7002052D532DC7BC
:102FE500F582852D83EBF0052EE52E7002052D5318
:102FF5002DC790634163A201852D83852E8263A22F
:10300500017F061225557406252EF52EE4352DF57E
:103015002D852A83852B8263A201852D83852E82AA
:1030250063A201AF2C1225557408252CF52CFFE45D
:10303500FCFDFEE5322FF532EE3531F531ED35305B
:10304500F530EC352FF52F908040E52FF0A3E530D6
:10305500F0A3E531F0A3E532F09080007420F0AFE5
:0D30650032AE31AD30AC2F906A8012209653
:01307200223B
:023203008F3FFB
:10320500E4F540F541908000E030E5110541E541E8
:1032150070020540D39488E540941340E8908000FF
:10322500E020E579906A80E0FCA3E0FDA3E0FEA341
:10323500E0F5458E448D438C42E545FFE544540752
:10324500FEE42FF541EE34C0F5409062B763A2016C
:1032550085408385418263A201AF3F122555E4FC79
:10326500FDFEE545253FF545EE3544F544ED354391
:10327500F543EC3542F542908040E542F0A3E54345
:10328500F0A3E544F0A3E545F09080007420F0AF8D
:0D32950045AE44AD43AC42906A80122096D5
:0132A2002209
:062E85008E2A8F2BAB0525
:102E8B00E4F52CF52D908000E030E511052DE52DB6
:102E9B007002052CD39488E52C941340E8908000A5
:102EAB00E030E503022F7E906A80E0FCA3E0FDA3F7
:102EBB00E0FEA3E0F5318E308D2F8C2EE531FFE552
:102ECB00305407FEE42FF52DEE34C0F52C852D8202
:102EDB00F5837423F0052DE52D7002052C532CC7BB
:102EEB00F582852C83EBF0052DE52D7002052C90DA
:102EFB00634163A201852C83852D8263A2017F062A
:102F0B001225557406252DF52DE4352CF52C532C57
:102F1B00C7E52A852D82852C83F0052DE52D7002C2
:102F2B00052C532CC7F582852C83E52BF0052DE55D
:102F3B002D7002052C532CC7E531240AF531E435ED
:102F4B0030F530E4352FF52FE4352EF52E908040FB
:102F5B00E52EF0A3E52FF0A3E530F0A3E531F090DB
:102F6B0080007420F0AF31AE30AD2FAC2E906A8064
:032F7B001220968B
:012F7E002230
:103CB700E5D220E0FBC2AF438E2075D2028F828E01
:0B3CC70083E0FFE4F5D2538EDFD2AFA4
:013CD20022CF
:103CED00E5D220E0FBC2AF43D2028F828E83EDF08E
:093CFD0075D25063D250D2AF22FF
:10366200E4FDED2401FFE433FE123CB774392DF57D
:1036720082E43463F583EFF00DBD3FE6E4FDED2413
:103682007FFFE433FE123CB7742F2DF582E43461E0
:10369200F583EFF0742F2DF582E43461F583E07049
:1036A2001B742F2DF582E43461F5837420F074309D
:1036B2002DF582E43461F583E4F080040DBD80BE13
:1036C200E49061AEF0FDEDFF7E00123CB774AF2DC9
:0D36D200F582E43461F583EFF00DBDFEE9F3
:0136DF0022C8
:023BDC008B2A32
:103BDE00A2AF9210C2AF85A22B53A2FE8E838F820C
:103BEE0005A28C838D8274091225DFE52A53A2FE6D
:103BFE0043A2201225E153A2DF852BA2A21092AF81
:013C0E00FFB6
:013C0F002292
:103C7E00A2AF9210C2AF8C838D82EF1225DF43A2CA
:0C3C8E00201225E153A2DFA21092AFFF2C
:013C9A002207
:023C36008F25D8
:103C3800A2AF9210C2AFE4F5838D8274061225DF1D
:103C4800E52543A2201225E153A2DFA21092AF7FFF
:013C5800016A
:013C59002248
:023C5A008F25B4
:103C5C00A2AF9210C2AFE4F5838D82740A1225DFF5
:103C6C00E52543A2201225E153A2DFA21092AF7FDB
:013C7C000146
:013C7D002224
:10240800A907E7FFA805EF93C3966008403B74FC53
:102418002FFF80F00F08EF93C3966008402B74FBE2
:102428002FFF80E00F08EF93C3966008401B74FAF3
:102438002FFF80D00F08EF93D3966008400B74F9F4
:102448002FFF80C01F1F1F1F1FEF54FEF80303F745
:10245800E893FC08E893FD08E893FE08E893FF2258
:1024680009E993C39D6008402974FB29F980F109A3
:10247800E993C39E6008401A74FA29F980E209E9D1
:1024880093D39F6008400B74F929F980D31919195F
:102498001919E9C313C313FF22740093F8ECC39806
:1024A8004024701F740193F8EDC398401970147498
:0E24B8000293F8EEC398400E7009740393F877
:1024C600EFC39840037F00227F0122EDF8E6F00873
:1024D600A3DFFA22EDF8E0F608A3DFFA22E0A36311
:1024E600A201F0A363A201DFF475A2002263A20198
:1024F600F0A363A20122E0A363A201F0A363A201F9
:10250600E0A363A201F0A363A201E463A201F0A326
:1025160063A201DFE175A20022E0A363A2016DFEC2
:10252600936CFDEE058393FC158363A201DFEA75C8
:10253600A200227F00E493A363A201F00F600CA324
:10254600E583C2E3F58363A20180EA75A20022E077
:10255600A363A201F0A3E583C2E3F58363A201DFCF
:10256600EE75A20022E0A363A201F0A3E583C2E414
:10257600D2E3F58363A201DFEC75A20022E0A36338
:10258600A201F0A3E58344F8C2E5F58363A201DF67
:10259600EC75A20022E583C2E3F583E0A363A20102
:1025A600F0A363A201DFEE75A20022E583C2E4D2A6
:0A25B600E3F583E0A363A201F0A3A4
:1025C00063A201DFEC75A20022E58344F8F583E005
:1025D000A363A201F0A363A201DFEE75A20022F9BA
:1025E00022C002C004C00612FFF0D006D004D00200
:0125F00022C8
:1013CE003E2A2C312CCFE0F0E0ECE5F2F0FB20F8D9
:1013DE00E8EDFB2043414E0A003E4C2C6B30312C85
:1013EE0025732C43EAEEF0EEF1F2FC20EDE020F84E
:1013FE00E8EDE52043414E2C30202D20353030EAEB
:10140E00E1283530EC292C31202D203530EAE12829
:10141E00353030EC290A0030202D20353030EAE10D
:10142E00283530EC290031202D203530EAE12835E1
:10143E003030EC29003E2A2C312CCFE0F0E0ECE5E8
:10144E00F2F0FB20EFF0EEF2EEEAEEEBE0204D4F85
:10145E00444255530A003E4C2C4930312C256C75B4
:10146E002CD1EAEEF0EEF1F2FC20EEE1ECE5EDE04F
:10147E002C343830302C393630302C313932303043
:10148E000A003E532C4931322C2562752CC0E4F0F3
:10149E00E5F120E1EBEEEAE020D2C8D220EDE0202B
:1014AE00F8E8EDE50A003E532C6D2562752C256299
:1014BE00752D25752D2562752D2562752CC7E0EFCE
:1014CE00F0EEF1202562752028B9CFF02DD0E5E39E
:1014DE002DCAEEEB2DD2E8EF290A003E532C5630E2
:1014EE00382C2562752CC8EDF2E5F0E2E0EB20EE2B
:1014FE00EFF0EEF1E0282A3130ECF1290A003C2120
:10150E00003C6B30313D003C4930313D003C4931AF
:10151E00323D003C5630383D002043616E457247E7
:10152E00495400200A002043616E457272434821DF
:10153E00000A00CEF2E2E5F23A00CEF8E8E1EAE087
:10154E0020CAD12100CEF8E8E1EAE020E0E4F0E59F
:10155E00F1E02100CEF8E8E1EAE020F2E8EFE02148
:10156E0000CEF8E8E1EAE020E4EBE8EDFB21000A2A
:10157E00C7E0EFF0EEF13A003C6D303D00000000A8
:10158E003C6D313D000000003C6D323D000000001E
:10159E003C6D333D000000003C6D343D000000000A
:1015AE003C6D353D000000003C6D363D00000000F6
:1015BE003C6D373D000000003C6D383D00000000E2
:1015CE003C6D393D000000003C6D31303D000000A7
:1015DE003C6D31313D0000003C6D31323D0000006C
:1015EE003C6D31333D0000003C6D31343D00000058
:1015FE003C6D31353D00000000C1814001C080418D
:10160E0001C0804100C1814001C0804100C18140C4
:10161E0000C1814001C0804101C0804100C18140B4
:10162E0000C1814001C0804100C1814001C08041A4
:10163E0001C0804100C1814001C0804100C1814094
:10164E0000C1814001C0804100C1814001C0804184
:10165E0001C0804100C1814000C1814001C0804174
:10166E0001C0804100C1814001C0804100C1814064
:10167E0000C1814001C0804101C0804100C1814054
:10168E0000C1814001C0804100C1814001C0804144
:10169E0001C0804100C1814000C1814001C0804134
:1016AE0001C0804100C1814001C0804100C1814024
:1016BE0000C1814001C0804100C1814001C0804114
:1016CE0001C0804100C1814001C0804100C1814004
:1016DE0000C1814001C0804101C0804100C18140F4
:1016EE0000C1814001C0804100C1814001C08041E4
:1016FE0001C0804100C1814000C0C101C30302C2CC
:10170E00C60607C705C5C404CC0C0DCD0FCFCE0E33
:10171E000ACACB0BC90908C8D81819D91BDBDA1AA3
:10172E001EDEDF1FDD1D1CDC14D4D515D71716D613
:10173E00D21213D311D1D010F03031F133F3F23283
:10174E0036F6F737F53534F43CFCFD3DFF3F3EFEF3
:10175E00FA3A3BFB39F9F83828E8E929EB2B2AEA63
:10176E00EE2E2FEF2DEDEC2CE42425E527E7E626D3
:10177E0022E2E323E12120E0A06061A163A3A26243
:10178E0066A6A767A56564A46CACAD6DAF6F6EAEB3
:10179E00AA6A6BAB69A9A86878B8B979BB7B7ABA23
:1017AE00BE7E7FBF7DBDBC7CB47475B577B7B67693
:1017BE0072B2B373B17170B0509091519353529203
:1017CE0096565797559594549C5C5D9D5F9F9E5E73
:1017DE005A9A9B5B99595898884849894B8B8A4AE3
:1017EE004E8E8F4F8D4D4C8C448485458747468653
:0817FE008242438341818040D7
:103CA10052668F00000000000000000000000000CC
:053CB10000000000000E
:013D1D002283
:030023000238C6DA
:1038C600C0E0C083C082C0D075D01830982CE55CAB
:1038D60025E9F5EB30D709E55B25F904F5FB80060C
:1038E600E55B25F9F5FBD29174582558F582E43449
:1038F60069F583E599F00558C29830992BE559C3C7
:1039060095575015D290AF59055974582FF582E442
:10391600346AF583E0F599800DAF578F59EF60064D
:103926000559D296C290C299D0D0D082D083D0E029
:01393600325E
:103C1000C2A9438902758C48758A4875D90475DB39
:103C20004875DC4875DD4875DE48E4F5E9F5F9C20C
:063C3000D9D28CD2DE2285
:102C81007BFF7A1379CE121C9D9068B1E0701475A8
:102C91002EFF752F147530257BFF7A1379E7121CEF
:102CA1009D8012752EFF752F147530347BFF7A13BA
:102CB10079E7121C9D7BFF7A147943121C9D906A5F
:102CC1007AE0FEA3E0FFC3E49FFFE49EFEAB07FAB8
:102CD1003395E0F9F87F007E8C7D0A7C00121FE5B8
:102CE1008F318E308D2F8C2E7BFF7A147964121CDC
:102CF1009D7BFF7A1479909068B2E0F52E121C9DAD
:102D0100E4F52A7BFF7A1479B4852A2EE52AFD336E
:102D110095E0FC74C52DF58274683CF583E0F52FD0
:102D2100AF2AEF3395E0FEEF25E0FFEE33FE74D6D8
:102D31002FF58274683EF583E0F530A3E0F5317438
:102D4100F62DF58274683CF583E0F532AF2AEF3356
:102D510095E0FE74072FF58274693EF583E0F53343
:102D6100E52A04F534121C9D052AC3E52A648094E2
:102D71009040907BFF7A1479E9906A79E0F52E1200
:022D81001C9D97
:012D8300222D
:10221A007E157F0C123459EF4E70037F0122E49031
:10222A0068B1F07E157F0F123459EF4E601B123CD5
:10223A00D38F25E525B431069068B1740AF0E525F7
:10224A00B432069068B17464F07E157F1512345961
:10225A00EF4E6023123A63A804A905AA06AB077FCA
:10226A00007E8C7D0A7C00121FE5122077906A7A24
:10227A00EEF0A3EFF0800A906A7A74FFF0A374B8C4
:10228A00F07E157F1B123459EF4E600A123A6390A2
:10229A0068B2EFF08005E49068B2F07E157F2112F3
:1022AA003459EF4E600D123A63906A78EEF0A3EF5C
:1022BA00F08009906A78E4F0A37464F0906A78E098
:1022CA00FEA3E0FF7C007D64121F978E5B8F5CE4A7
:1022DA00F556F525E525FD3395E0FC74C52DF58207
:1022EA0074683CF583E4F0E525FB3395E0FAEB25C9
:1022FA00E0FFEA33FE74D62FF58274683EF583E474
:10230A00F0A3F074F62DF58274683CF583E4F0AF1F
:10231A0025EF3395E0FE74072FF58274693EF58345
:10232A00E4F074B32FF58274683EF583E4F074A187
:10233A002FF58274683EF583740FF0EBAE027803D2
:10234A00C333CE33CED8F92486F58274153EAF82D4
:10235A00FE123459EF4E70030223F4123A63E52554
:10236A00FD3395E0FC74C52DF58274683CF583EF66
:10237A00F074C52DF58274683CF583E0606C123AFE
:10238A0063AD07AC06AF25EF3395E0FEEF25E0FF1E
:10239A00EE33FE74D62FF58274683EF583ECF0A313
:1023AA00EDF0123A63E525FD3395E0FC74F62DF560
:1023BA008274683CF583EFF0123A63E525FD3395A4
:1023CA00E0FC74072DF58274693CF583EFF074B371
:1023DA002DF58274683CF583E556F074F62DF58286
:1023EA0074683CF583E02556F5560525C3E5256452
:0D23FA0080949050030222DE7556FF7F0094
:0124070022B2
:1039370043AB01C2E8C2EAE4FFEFC454F0F5B1C3F8
:10394700EF64809488500575B3D08003E4F5B3E441
:10395700F5B275BCC8F5BDF5BE75BF7875C4FFF582
:10396700C5F5C675C778F5A3F5A3F5A3F5A3F5A324
:10397700F5A3F5A3F5A30FBF0EBF9068B1E0FF2530
:10398700E0F5B475B50C75B66C75A11275AB02751B
:08399700C13E75C3FF75C203B8
:01399F002205
:103A030075B180E4F5B3F5B28547BCE5485403FFCF
:103A130033333354F8FFE54854E04FFFE549C4130B
:103A230054074FF5BDE54933333354F8FFE54AC432
:103A33001354074FF5BEE54A33333354F8F5BF85C6
:103A43004CA3854DA3854EA3854FA38550A38551D4
:103A5300A38552A38553A3E54B540F2450F5B322FA
:102A7000E59B541F6020200B1A7E157F27122D84A2
:102A8000E59B541FFF7E007D03122E857E157F314E
:102A9000122D84E4F59BE5BA30E008E4F5B375B196
:102AA00080F5B2E5CFF47003022B7A752901E4F5C5
:102AB00028E5CFF455297003022B68E528C454F0AB
:102AC000F5B1E5B2547F6420706FE5B3540FF54B58
:102AD00085BC47E5BD541FFF131313541FFFE5BD0D
:102AE00054E044184FF548E5BDC43354E0FFE5BE5B
:102AF000131313541F4FF549E5BEC43354E0FFE5EB
:102B0000BF131313541F4FF54A85A34C85A34D855E
:102B1000A34E85A34F85A35085A35185A35285A3BA
:102B200053E4F5B2E547547EB5470575B3508003CD
:102B300075B3D0E54B2405FF22E5B2549F602320F6
:102B40000B207E157F34122D84AFB27E007D0312E0
:102B50002E85AFB37E007D03122E857E157F3F123A
:102B60002D84E4F5B275B3D0E52925E0F5290528D3
:0C2B7000E528C394085003022AB17F003E
:012B7C002236
:1036E000C219E4F558F50BD296C21AF557F559FFF1
:1036F0007F40906918E4F0A3DFFC7F40E4F55AF5C1
:103700005E12221A123937C2ADE4F5C9D2CDD2CC3D
:10371000C2C9C2CAF5CDF5CC906A7AE0F5CBA3E078
:10372000F5CA85CBCD85CACCE4F598D29E438740B7
:10373000C29FC2ACC298C29975B81075B710D2CAF0
:10374000D29CD2AC123C10C2D9E5E92464F5EB302E
:0B375000D706E5F904F5FB2285F9FB24
:01375B00224B
:013D1E002282
:013D1F002281
:05001E00D29CD2AC22CF
:013D20002280
:063B6000AC05AB07AA064C
:103B660090690674FFF0906917F0AF041CEF602DA2
:103B76000BEBAE0270010A14F5828E83E0FF9069AA
:103B860006E06FFF90160693FE906917E06E906947
:0D3B960006F0EF90170693906917F080CDB0
:013BA30022FF
:1038500074C52556F582E43468F583E0906A58F023
:1038600074072556F582E43469F583E0906A59F0CF
:10387000E55625E024D6F582E43468F583E0FCA320
:10388000E0FDEC906A5AF0A3EDF0E4A3F074F625A5
:1038900056F582E43468F583E0906A5DF07E6A7FD5
:1038A000587D06123B60906906E0906A5EF0906970
:1038B00017E0906A5FF0E4F559755708C296C2990F
:0638C0002099FDD29922BF
:10333F00E55EC394404003E4F55E7418255EF582A4
:10334F00E43469F583E0FF30E16F7418255EF58290
:10335F00E43469F583EF54FDF0E4906478F0A374DE
:10336F000DF090667CE090647AF0A37419F0A3746A
:10337F0048F0A37479F0E55E131313541FFF9068A0
:10338F00B2E02F90647EF0E55E540725E025E0243F
:10339F0080A3F0A37408F0F5F0E55EA424A1F582F4
:1033AF00E5F03466F58363A20190648163A2017F27
:0E33BF00081224E3055E7F0122055E7F0022D6
:013D2100227F
:101806007418255AF582E43469F583E020E0020570
:101816005AE55AC394404003E4F55A122A70EF6021
:1018260069E54A640F70639068B2E0FF6549705AD3
:101836007418255AF582E43469F583E0FE30E04AEF
:101846007418255AF582E43469F583EE54FEF07572
:101856004748754879E55A131313541FFEEF2EF5C2
:1018660049E55A540725E025E02480F54A754B08DA
:1018760075F008E55AA424A1F582E5F03466F583EF
:101886007D4C7F081224DA123A03300249C20290D4
:1018960068C4E004F070069068C3E004F0D3906872
:1018A600C4E094B89068C3E0940B402AE4F0A3F037
:1018B600F52574182525F582E43469F583E030E2D0
:1018C6000E74182525F582E43469F5837403F00552
:1018D60025E525B440DC20D903021C3AE557700300
:1018E600021BCBE558D394005003021AB5C291856A
:1018F600585D74B32556F582E43468F583E075F0D7
:1019060002A485F026F527E4F5587E697F5890698C
:101916005AE02405FD123B60200B127E157F411212
:101926002D847E697F58E4FBAD5D122F7F90691789
:10193600E0FF906906E04F6010300B03021BCB7E80
:10194600157F48122D84021BCB74C52556F582E4FB
:101956003468F583E0FF906958E06F6010300B0340
:10196600021BCB7E157F53122D84021BCB740725D9
:1019760056F582E43469F583E0FF906959E06F60BB
:1019860010300B03021BCB7E157F62122D84021BC7
:10199600CB74F62556F582E43468F583E075F002DB
:1019A600A4FF90695AE06F7002E5F06010300B03F7
:1019B600021BCB7E157F6F122D84021BCB74A125D3
:1019C60056F582E43468F583E4F0F52590695AE02B
:1019D600FFE525C39F4003021BCB74A12527F58293
:1019E60074663526F583E0FF745C2525F582E434BC
:1019F60069F583E0FEEF6E602774A12527F58274F2
:101A0600663526F583EEF0E527AE267803CEC313BA
:101A1600CE13D8F92418F58274693EF5837407F05D
:101A2600E527AE267803CEC313CE13D8F92418F5CE
:101A36008274693EF583E04404F00527E5277002C9
:101A4600052624A1F58274663526F583E0FF745BCE
:101A56002525F582E43469F583E0FEEF6E60277490
:101A6600A12527F58274663526F583EEF0E527AEC7
:101A7600267803CEC313CE13D8F92418F5827469D9
:101A86003EF5837407F0E527AE267803CEC313CE62
:101A960013D8F92418F58274693EF583E04404F0FE
:101AA6000527E52770020526052505250219D274A6
:101AB600A12556F582E43468F583E004F074A12587
:101AC60056F582E43468F583E0D3940A5003021B8A
:101AD600CB74A12556F582E43468F5837405F07459
:101AE600B32556F582E43468F583E075F002A485E3
:101AF600F026F527E4F52574F62556F582E43468D4
:101B0600F583E0FFE525C39F4003021BCB74A125A7
:101B160027F58274663526F583E0F4602874A125DE
:101B260027F58274663526F58374FFF0E527AE2621
:101B36007803CEC313CE13D8F92418F58274693E00
:101B4600F5837407F0E527AE267803CEC313CE13CC
:101B5600D8F92418F58274693EF583E04404F0054B
:101B660027E5277002052624A1F58274663526F539
:101B760083E0647F602874A12527F5827466352684
:101B8600F583747FF0E527AE267803CEC313CE1314
:101B9600D8F92418F58274693EF5837407F0E527B1
:101BA600AE267803CEC313CE13D8F92418F5827463
:101BB600693EF583E04404F00527E5277002052613
:101BC6000525021AFD0556E4F557E556C39410504F
:101BD6006074C52556F582E43468F583E060557473
:101BE600F62556F582E43468F583E06047200B0756
:101BF6007E157F7D122D84C2D9123850E55C24E80B
:101C060025E9F5EB30D70FE55C24E8E55B340325E1
:101C1600F904F5FB800CE55C24E8E55B340325F963
:101C2600F5FB200B0F7E6A7F58E4FB7D08122F7FA1
:041C3600227556FFBE
:011C3A002287
:033D1A007F002205
:1033D9000208A4E493A3F8E493A34003F68001F25E
:1033E90008DFF48029E493A3F85407240CC8C333F5
:1033F900C4540F4420C8834004F456800146F6DFC4
:10340900E4800B0102040810204080903C9BE47E7C
:10341900019360BCA3FF543F30E509541FFEE493B8
:10342900A360010ECF54C025E060A840B8E493A37F
:10343900FAE493A3F8E493A3C8C582C8CAC583CAAA
:10344900F0A3C8C582C8CAC583CADFE9DEE780BE62
:013CB600000D
:101F9700EF8DF0A4A8F0CF8CF0A428CE8DF0A42E5E
:021FA700FE2218
:101FA90075F008758200EF2FFFEE33FECD33CDCCEF
:101FB90033CCC58233C5829BED9AEC99E582984072
:101FC9000CF582EE9BFEED9AFDEC99FC0FD5F0D64F
:101FD900E4CEFBE4CDFAE4CCF9A88222B800C1B979
:101FE9000059BA002DEC8BF084CFCECDFCE5F0CBB7
:101FF900F97818EF2FFFEE33FEED33FDEC33FCEBF0
:1020090033FB10D703994004EB99FB0FD8E5E4F9AA
:10201900FA227818EF2FFFEE33FEED33FDEC33FC97
:10202900C933C910D7059BE99A4007EC9BFCE99A8B
:10203900F90FD8E0E4C9FAE4CCFB2275F010EF2FD0
:10204900FFEE33FEED33FDCC33CCC833C810D707D0
:102059009BEC9AE899400AED9BFDEC9AFCE899F80B
:0E2069000FD5F0DAE4CDFBE4CCFAE4C8F9229E
:0E207700C3E49FFFE49EFEE49DFDE49CFC227A
:10208500EB9FF5F0EA9E42F0E99D42F0E89C45F0B1
:012095002228
:0C209600ECF0A3EDF0A3EEF0A3EFF022BD
:1020A200A8828583F0D083D0821220B91220B9127F
:1020B20020B91220B9E473E493A3C583C5F0C583A4
:1020C200C8C582C8F0A3C583C5F0C583C8C582C888
:0120D20022EB
:101C3B00E53A242EF8E6053A22782B301702782E57
:101C4B00E475F00112217A0220D32010EB7F2ED203
:101C5B00108018EF540F2490D43440D4FF30140B61
:101C6B00EF24BFB41A0050032461FFE53B6002155B
:101C7B003B053EE53E7002053D30170D782BE475B4
:101C8B00F00112217AEF022119023B197403D217CA
:101C9B008003E4C217F53A8B2B8A2C892DE4F53B94
:101CAB00F53DF53EE53B60077F20121C7680F57510
:101CBB003CFFC211C210C212C213C215C216C21807
:101CCB00121C44FF700D3017057F00121C87AF3EAE
:101CDB00AE3D22B4255FC2D5C214121C44FF24D0E2
:101CEB00B40A00501A75F00A783B30D50508B6FFD8
:101CFB000106C6A426F620D5047002D21380D9247F
:101D0B00CFB41A00EF5004C2E5D214021E87D211D1
:101D1B0080C6D21080C0D21280BCD2D580BAD21568
:101D2B0080B47F20121C762012077401B53B004053
:101D3B00F1121C3BFF121C76021CAFD218D216807C
:101D4B0095121C3BFB121C3BFA121C3BF94A4B70C5
:101D5B000679587A1F7BFF20122EE53B602A7E0006
:101D6B008E827583001220EC60060EEE653C70F0DF
:101D7B00C2D5EBC0E0EAC0E0E9C0E0EE121ECED067
:101D8B00E0F9D0E0FAD0E0FB1220D3FF60AAEBC061
:101D9B00E0EAC0E0E9C0E0121C76D0E02401F9D003
:101DAB00E03400FAD0E0FBE53C0460DCD53CD980A4
:101DBB00877BFF7A1E79CAD212809C7910800279B8
:101DCB0008C216C2188008D2D5790A8004790AC2D3
:101DDB00D5E53C047002F53CE4FAFDFEFF121C3B1A
:101DEB00FC7B08201113121C3BFD7B1030100A12D8
:101DFB001C3BFE121C3BFF7B20EC3382D592D55053
:101E0B0013C3E43010069FFFE49EFEE42011039DF4
:101E1B00FDE49CFCE4CBF8C211EC700CCFCECDCC26
:101E2B00E824F8F870F38017C3EF33FFEE33FEEDC1
:101E3B0033FDEC33FCEB33FB994002FB0FD8E9EBA2
:101E4B00301105F8D0E0C448B211C0E00AEC4D4E99
:101E5B004F78207B0070C2EAB53C0040BCC0E0125A
:101E6B001ED0D0F0D0E0201104C4C0E0C4B211C029
:101E7B00F0121C5FD0F0D5F0EB021CAF1221D91D74
:101E8B004C531DC6581D1D4C1D19421DCA4F1DD24A
:0F1E9B00441DD2491D32431DD8551DBC461DBCE8
:101EAA00451DBC471F78501D212D1D252E1D482B71
:101EBA001D29231D46201F612A1CE14800001D40E0
:101ECA003F3F3F00790AA2D5201314301509B910F3
:101EDA00020404B9080104A2D52016025001042004
:101EEA0012689212B53B005034C0E07F20301319BB
:101EFA007F30A21272167215500F121F27C212C219
:101F0A0016C215C2187F30800F301503E9C0E012DF
:101F1A001C76301503D0E0F9D0E0B53BCC3015176C
:101F2A007F30B9100C121C767F583014077F7880E6
:101F3A0003B90803121C763012057F2D021C767F26
:101F4A00202018F87F2B2016F322921280CF286EB9
:101F5A00756C6C2900D211121C3B3011F8C2117831
:101F6A003B30D50108F6021CE12D50434958121C9A
:101F7A003B2403B405004001E4901F7393121C67CD
:0D1F8A00743A121C67D213753B04021DC689
:1025F1008B2A8A2B892CE4F536F535F534F533F53C
:1026010031F532E52E452F452D6012EBC0E0EAC0D1
:10261100E0E9C0E0AB2DAA2EA92F12218AAB2A0531
:102621002CE52CAA2B7002052B14F91220D3F537B7
:10263100C394094007E537D3940D40E1E5376420A1
:1026410060DBE537B42D054332038016E537B42B43
:1026510005433201800C74FF252CF52C74FF352BBA
:10266100F52BE53060046410703FAB2AAA2BA92C2E
:102671001220D364306009E530702E75300A80294C
:102681009000011220ECFF64786004EFB45813430A
:1026910032017530107402252CF52CE4352BF52B05
:1026A1008007E5307003753008AB2A052CE52CAAAC
:1026B1002B7002052B14F91220D3F537C394614016
:1026C1000AE537D3947A50035337DF74D02537F5B1
:1026D10037C3940A400CE5379411406D74F92537DE
:1026E100F537E537D39530506043320185363B8568
:1026F100353A853439853338AF307E00E4FCFDABA3
:1027010036AA35A934A83312212BC8ECC8C9EDC9A2
:10271100CAEECACBEFCBE4FCFDFEEB2537F536EE76
:102721003AF535ED39F534EC38F533AF36AE35AD34
:1027310034FCAB3BAA3AA939A838D31220855003FF
:102741000226AA4332040226AAE53220E003E480ED
:102751002DE52E452F452D601EAB2AE52C24FFF9D2
:10276100E52B34FFFAEBC0E0EAC0E0E9C0E0AB2DB5
:10277100AA2EA92F12218AE53230E20774FFFFFE4B
:10278100FDFC22E532AF36AE35AD34AC3330E1037A
:042791000220772289
:1020D300BB010689828A83E0225002E722BBFE020B
:0920E300E32289828A83E493223E
:1020EC00BB010CE58229F582E5833AF583E02250A9
:1020FC0006E92582F8E622BBFE06E92582F8E222F3
:0D210C00E58229F582E5833AF583E493220C
:10211900BB010689828A83F0225002F722BBFE01A5
:02212900F3229F
:10212B00E88FF0A4CC8BF0A42CFCE98EF0A42CFC53
:10213B008AF0EDA42CFCEA8EF0A4CDA8F08BF0A4D1
:10214B002DCC3825F0FDE98FF0A42CCD35F0FCEB30
:10215B008EF0A4FEA9F0EB8FF0A4CFC5F02ECD39F5
:0F216B00FEE43CFCEAA42DCE35F0FDE43CFC2262
:10217A00FAE6FB0808E6F925F0F618E6CA3AF62266
:10218A00BB011A89828A83D0F0D0E0F8D0E0F9D076
:10219A00E0FAD0E0FBE8C0E0C0F00222085016E9FD
:1021AA00F8D083D082D0E0F9D0E0FAD0E0FBC08248
:1021BA00C0830221FFBBFE16E9F8D083D082D0E0AB
:0F21CA00F9D0E0FAD0E0FBC082C08302221122DC
:1021D900D083D082F8E4937012740193700DA3A395
:1021E90093F8740193F5828883E4737402936860A9
:0621F900EFA3A3A380DFA9
:0921FF00EBF608EAF608E9F62205
:09220800EBF0A3EAF0A3E9F022D7
:09221100EBF208EAF208E9F222FE
:00000001FF
